:020000040000FA
:10000000AF2A000000000000092B000008000830A3
:10001000FC002330FD00FD0B0B28FC0B0B28080017
:100020001030FD00FD0B122800000800831603139A
:10003000A41B1D28831286131F288312861783167C
:10004000241B2528831206132728831206178316DC
:10005000A41A2D28831286122F288312861683163F
:10006000241A3528831206123728831206166918B7
:100070003B2805143C28051085140520851083169F
:10008000A4194528831286134728831286178316DE
:1000900024194D28831206134F288312061783163E
:1000A000A4185528831286125728831286168316A1
:1000B00024185D28831206125F2883120616691819
:1000C0006328051464280510851405208510691C13
:1000D0006B2807206C281020080083120313691076
:1000E00083162308A400162069140800710DF80D6A
:1000F000F90D7408F8027508031C750FF902F00D6C
:10010000F10D0F30FC00710DF80DF90D7408701C25
:100110008F28F8027508031C750FF9029428F80758
:1001200075080318750FF907F00DF10DFC0B832806
:100130007018A0287408F80775080318750FF907D8
:1001400000000800B428803083160313A000C728DD
:10015000C030A000C7289430A000C728D430A00029
:10016000C7288030A000C728831603132008013A4F
:100170000319A3282008023A0319A8282008033AE3
:100180000319AB282008043A0319AE28B12821032B
:10019000F0002008F0077008A0007008A4001620E6
:1001A0006910EF016F088316220784000008031905
:1001B000E32883126F088316220784000008A30037
:1001C0006D20EF0AD22883126914080083120313EA
:1001D00063088A0062088200080083120313FD018D
:1001E000F901F801710870040319003471087506EB
:1001F000FA00FA1BFD09FB01F51F0329F409F509B3
:10020000F40A0319F50AF11F0A29F009F109F00AA5
:100210000319F10A71087504FA00FA1B1F297620E8
:100220007B183229FD1F0034F009F109F00A031987
:10023000F10AF809F909F80A0319F90A0034F51F57
:100240002E29F11B2A297108F9007008F800F10124
:10025000F0011229F101F001F00A0034F109F0096E
:10026000FB0A0F29F80A0319F90A74087802031D1A
:10027000122975087902031D1229F901F801F00A03
:100280000319F10AF11F12290000FF34080059294F
:10029000803083160313A0006C29C030A0006C29A5
:1002A0009430A0006C29D430A0006C298030A000CC
:1002B0006C29831603132008013A031948292008E2
:1002C000023A03194D292008033A0319502920083E
:1002D000043A0319532956292103F0002008F00796
:1002E0007008A0008312691470088316A4001620F9
:1002F000691083162208A4001620691408008312CE
:10030000031385150130AC0001308316A4001620BC
:1003100001308316A0000130A1002830A200A220E5
:1003200002308316A0000130A1002D30A200A220CF
:1003300080308316810090308B008312E5016B08BA
:10034000650203180D2A65086B02ED00EE01031C1F
:10035000EE030A30F4000030F5006D08F0006E087E
:10036000F100ED207808F0007908F1007008EC0049
:100370000A30F4000030F5006D08F0006E08F1005E
:10038000ED2002308316A0000C30A1003030700741
:10039000A200472102308316A0000D30A1003030AA
:1003A00083126C078316A20047210130E600063055
:1003B000FB001330FC00AD30FD00FD0BDD29FC0B14
:1003C000DD29FB0BDD2900000000E60A66083C3C45
:1003D000031CEF296708003A031DEF29D729670896
:1003E00003190B2A85110330FB008A30FC005530BD
:1003F000FD00FD0BF929FC0BF929FB0BF929000085
:10040000000001308316A0000130A1002330A200BB
:10041000A2208B010D2AE50A9F298511AC01A101BB
:10042000A0010130E7000800831203137008F100F7
:10043000F0010830FC007108F40C0318232AFC0BAF
:100440001C2AF10100340310282AF40C0318F107C8
:10045000F10CF00CFC0B252A0800E6208A110A1288
:100460008000840AE20A0319E30AF003031D2D2A1F
:100470000800831603138510051006128612061352
:100480008613831285100510861306138612061232
:1004900007200720072086160616851405208510DC
:1004A0000720851405208510072085140520851058
:1004B00007200612851405208510072085140520C5
:1004C000851086128617851405208510072086134F
:1004D0000616851405208510061285140520851042
:1004E0000720851405208510061685140520851023
:1004F0000720061285140520851086170617861614
:10050000061685140520851007206914080083123B
:100510000313220A840030302107F00070088000A5
:1005200030302007F000220884007008800002307C
:100530008316A0000B30A100831222088316A200AC
:10054000A22008000230FB008630FC009930FD003C
:10055000FD0BA82AFC0BA82AFB0BA82A08005E2387
:100560000730831203139F040F3083168600F03088
:100570008500831285113922E70101308316A4001A
:1005800016200C308316A400162001308316A0001C
:100590000130A1003E30A200A22002308316A0004C
:1005A0000130A1004E30A200A22087228618E02A46
:1005B000A222A10A21080A3A031DDF2AA1018722EB
:1005C0000619EA2AA222A00A20080A3A031DE92AEB
:1005D000A00187220618FE2AA2222008F0000A3075
:1005E000F400142221087007F1007108E40071087A
:1005F000003C0318FE2A6408EB007F2167080319FA
:10060000022BBC2AD62A032BFF3FFF3FFF3FFF3FB1
:10061000FF3FFF00030E8301EA000A08E8008A0199
:100620008B1C152B0130E7008B1068088A006A0EBE
:100630008300FF0E7F0E0900003400345F34203445
:100640004F3446344634003420344F344E34003472
:100650000034413470346F346D3465346E346F342B
:1006600075346E343A342034203420346D34693497
:100670006E34003450346F3477346534723443341C
:100680006934723463347534693474342E346534A7
:100690007534003450346F347334613420346D3425
:1006A00069346E343A3420342034203420346D34AC
:1006B00069346E34003430343034003420308400F7
:1006C000423083120313F0001C30E2000330E300D9
:1006D0002D220800FF3FFF3FFF3FFF3FFF3FFF3F4F
:1006E000FF3FFF3FFF3FFF3FFF3FFF3FFF3FFF3F1A
:1006F000FF3FFF3FFF3FFF3FFF3FFF3FFF3FFF3F0A
:10070000FF3FFF3FFF3FFF3FFF3FFF3FFF3FFF3FF9
:10071000FF3FFF3FFF3FFF3FFF3FFF3FFF3FFF3FE9
:04400E00693FFF3FC8
:00000001FF
